:1000000055C089C06EC06DC06CC06BC06AC069C08D
:1000100068C067C066C065C064C0B7C1F3C161C0D5
:1000200060C05FC05EC05DC05CC05BC05AC059C0EC
:1000300058C057C00902220001010080FA090400DB
:100040000001030000000921010100012221000735
:100050000581030800641201100100000008C016A9
:10006000DF050001010200010E037500730062004C
:1000700069003200630010036300650072006E00C7
:100080002E0063006800040309040600FF0901A1B3
:1000900001150026FF007508850195110900B202BF
:1000A00001850295830900B20201C00011241FBE20
:1000B000CFEFD4E0DEBFCDBF11E0A0E0B1E0ECECCB
:1000C000F7E102C005900D92A233B107D9F721E004
:1000D000A2E3B1E001C01D92A93FB207E1F76DD5DF
:1000E00073CB8ECFA82FB92F80E090E041E050EA8B
:1000F000609530E009C02D9182279795879510F083
:1001000084279527305EC8F36F5FA8F30895EADF70
:100110008D939D930895CF93CFB7CF93C3954B9B6A
:10012000E9F74B9B09C04B9B07C04B9B05C04B9B02
:1001300003C04B9B01C0A3C0DF93C091D601DD2754
:10014000C352DE4F4B9B02C0DF91EBCF2F930F9337
:100150001F9309B12FEF03FB20F94F933F9319B180
:100160004FEF012703FB21F93BE031C04E7F012F08
:1001700019B1216028C0102F4D7F2260000009B105
:1001800029C04B7F2460012F000019B12BC019B189
:10019000477F28602AC04F7E09B120612CC04F7D67
:1001A00019B120622FC04F7B09B1206432C04227B1
:1001B00009B149934FEF0000102713FB20F919B143
:1001C0001C70C9F1297F91F2012703FB21F909B1C4
:1001D000237F89F2315058F1102713FB22F919B10E
:1001E000277E79F2012703FB23F92F7C81F209B1E5
:1001F000102713FB24F92F7971F200C019B10127E0
:1002000003FB25F92F7359F200C009B1102713FB26
:1002100026F9223040F200C019B1012703FB27F96B
:10022000243028F64F77206819B10000F9CF11E08B
:100230001CBB002719C03B503195C31BD04011E0B7
:100240001CBB0881033CF9F00B34E9F02091D40188
:100250001981110F1213EDCF4A81441F093641F164
:100260000D3211F0013E29F70093DB013F914F91D0
:100270001F910F912F91DF91CCB3C0FD4FCFCF9144
:10028000CFBFCF9118952091DB01222379F31091F4
:10029000D901112369F534306AF13093D9012093E3
:1002A000D5011091D6013BE0311B3093D60122C01D
:1002B0000091D9010130E4F40AE54F7049F430911E
:1002C000010134FD19C000930101CDEBD1E018C04C
:1002D0003091C80134FD10C00093C801C9ECD1E0D1
:1002E0000FC02795A8F45150A9F4220F0000F9CFB0
:1002F0004AE503C042ED01C0432FC4E1D0E032E043
:100300001AB11C605B9A1AB90BB120E41CE05F9330
:10031000012756E00BB9279520F4515021F4220F04
:10032000F9CF012756E000003B5A0BB9D0F22795D0
:1003300028F4515029F4220F0000F9CF012756E08C
:1003400027950BB920F4515021F4220FF9CF012742
:1003500056E0299133230BB921F6037F1091DA017E
:10036000110FC651D0400BB911F01093D40111E018
:100370001CBB08601AB1137F402F437F5F9100C000
:1003800000C00BB91AB94BB971CF1F920F920FB6BB
:100390000F9211248F939F9380913201909133019A
:1003A00001969093330180933201809132019091B4
:1003B0003301069769F41092330110923201809153
:1003C000BB019091BC0101969093BC018093BB014D
:1003D0009F918F910F900FBE0F901F901895CF9304
:1003E000C62F880F07D1813021F42ED181E090E013
:1003F00007C086E639D18C2F37D126D180E090E036
:10040000CF9108951F920F920FB60F9211242F9340
:100410008F939F9380913701909138018F3F2FEFF9
:10042000920729F0019690933801809337018091CB
:100430003601882329F0809135018F5F8093350143
:100440009F918F912F910F900FBE0F901F90189535
:1004500082E080936E0084BD85B5856085BD84E7AC
:1004600087BD8BE886BDA99AEFE6F0E080818260C7
:1004700080830895CF93C82F909136019923A1F0DE
:10048000809135018B3018F0109235016AD090912F
:1004900036019230B9F018F4911149C005C093307B
:1004A00011F1943089F143C0C13009F043C082E0BA
:1004B0008093360181E090E074D010923801109260
:1004C000370138C08091370190913801C39790F17E
:1004D00083E080933601109238011092370181E059
:1004E00090E049D027C08091370190913801C3979F
:1004F00008F184E0809336011092380110923701A0
:1005000080E090E038D016C080913701909138019A
:10051000C39780F01092360180E090E026D01092D0
:1005200038011092370180E090E03BD003C082E0B8
:1005300080933601CF91089595B180E1892785B9DF
:100540000895892B11F02C9A08952C98089583B161
:10055000829581700895892B11F0429A08954298EE
:1005600008958BB180588BB90895892B11F05F9A4B
:1005700008955F980895892B11F0289A0895289876
:100580000895892B11F0299A08952998089583B127
:10059000869581700895892B11F02A9A08952A98DA
:1005A0000895892B11F05D9A08955D980895892B1F
:1005B00011F05E9A08955E98089589B186FB8827A8
:1005C00080F908951092B90084E38093B8000895EB
:1005D00080E790E0ECEBF0E006C024E02A95F1F72C
:1005E0000197009729F020812223BCF780E008952D
:1005F00081E00895CF93C82F94EA9093BC00E8DF80
:10060000811119C09091B900987F983011F0903104
:10061000A1F4C093BB0084E88093BC00D9DF8111B2
:100620000EC09091B900987F983151F081E09034DC
:1006300039F480E005C081E003C081E001C081E0C1
:10064000CF910895D7DF089584E98093BC0080E7B7
:10065000ECEBF0E005C094E09A95F1F7815019F0C9
:10066000908194FDF8CF08958093BB0084E8809337
:10067000BC00AEDF811108C09091B900987F81E085
:10068000983219F480E0089581E0089584EC809315
:10069000BC009EDF811104C08091BB0090E00895F2
:1006A0008FEF9FEF089584E88093BC0091DF811164
:1006B00004C08091BB0090E008958FEF9FEF0895F4
:1006C0001092C5008CE08093C400E0ECF0E08081E3
:1006D0008260808388E18093C1000895CF93C82F02
:1006E0008A3011F48DE0FADFE0ECF0E0908195FFC4
:1006F000FDCFC093C60080E090E0CF9108956F9247
:100700007F928F929F92AF92BF92CF92DF92EF92A1
:10071000FF920F931F93CF93DF938C0180918901F8
:1007200090918A01892B09F0C6C00F2EF9E38F2E14
:10073000F1E09F2EF02DC0ECD0E00F2EF6ECCF2E86
:10074000D12CF02D54010F2EF8E36F2EF1E07F2E07
:10075000F02D88818823ECF7888184FDBFC08881D3
:1007600083FDBFC0F60180818D3011F08A3061F4C5
:100770008AE0F4018083B801B1DF89E391E09093CE
:100780008A018093890197C0893039F090EE980FE3
:100790009F3520F0803AA8F001C080E2F8E88F167B
:1007A000F1E09F0621F4B80187E098DFD2CF740111
:1007B0009FEFE91AF90AF4018083B8018FDF47013E
:1007C000C8CF8231B9F130F4833009F48DC088305C
:1007D000E9F0BFCF873129F08F37C1F0853179F04B
:1007E000B8CFF9E38F16F1E09F0609F008F4B1CF16
:1007F000F40131978081803209F045C0AACF89E3A6
:10080000881681E0980609F048F5A3CF99E3891688
:1008100091E0990609F008F49CCFB80188E05EDF0A
:10082000B80180E25BDFB80188E058DFE1E08E1AB2
:1008300091088FCFB8018DE051DFF9E38F16F1E019
:100840009F0609F008F485CF7501B801F701819181
:100850007F0144DFE814F904C1F77BCFB80188E0D9
:100860003DDFB80180E23ADFB80188E037DFF1E030
:100870008F1A910889E3881681E0980679F7F301C9
:1008800031964F0166CFB80188E028DFB80180E2D9
:1008900025DFB80188E022DFF1E08F1A910889E3B3
:1008A000881681E0980609F454CFF40131978081CD
:1008B000803249F74ECFE0918901F0918A01CF0152
:1008C000019690938A018093890180818A3021F476
:1008D00010928A011092890190E008C08EEF9FEF7C
:1008E00005C08FEF9FEF02C08FEF9FEFDF91CF9199
:1008F0001F910F91FF90EF90DF90CF90BF90AF903E
:100900009F908F907F906F900895CF93DF93609129
:10091000D90163500AF4CFC02091D6018CE090E059
:10092000821B9109EC01C352DE4F8091D5018D32BB
:1009300009F0B0C0683009F0BCC083EC8093BD0101
:100940008AE58093010110928B018881807619F0ED
:10095000CE01F7D38BC09A811092C6018981811193
:1009600006C01092C70126EC31E082E07BC08530E2
:1009700031F49093DA0126EC31E080E073C08630E8
:1009800009F050C08B81813041F486E590E090936E
:10099000D8018093D70182E141C0823041F484E3E1
:1009A00090E09093D8018093D70182E237C08330E2
:1009B000F1F4911108C086E890E09093D8018093FB
:1009C000D70184E02BC0913041F486E790E090930A
:1009D000D8018093D70180E121C09230E1F488E60C
:1009E00090E09093D8018093D7018EE017C08132B8
:1009F00041F486E490E09093D8018093D70189E098
:100A00000DC0823251F48AE890E09093D80180932F
:100A1000D70181E203C080E001C080E090E49093C0
:100A20008B0124C0883099F0893031F49093DC0137
:100A300026EC31E080E016C08A3069F08B3079F422
:100A40008BE48093C90126EC31E080E00BC02CEDF3
:100A500031E081E007C026EC31E081E003C026EC04
:100A600031E080E03093D8012093D7018F3F41F4EB
:100A7000988199230CF48E8190E890938B0107C0A4
:100A80009F81911104C09E81981708F4892F80934B
:100A900000010FC080918B0188235CF4CE0109D343
:100AA0008F3F21F48EE18093010103C081111092E8
:100AB00000011092D9018091010184FF5AC08091F8
:100AC00000018F3F09F455C0C82F893008F0C8E0F5
:100AD0008C1B80930001EDEBF1E0908188E8892781
:100AE0008083CC2309F453C080918B01882334F494
:100AF0006C2F8EEB91E008D3C82F28C02091D7012E
:100B00003091D80186FF10C0AEEBB1E0F9018C2F17
:100B100094919D9331968150D9F72F5F3F4F8FEF7E
:100B20008C0F280F311D0EC0AEEBB1E0F9018C2FF8
:100B300091919D938150E1F72F5F3F4F8FEF8C0F85
:100B4000280F311D3093D8012093D701C93058F4B4
:100B50006C2F8EEB91E0DBDACC5FCC3040F48FEF82
:100B60008093000104C08FEF80930001CEE1C09319
:100B7000010189B18C7089F483E199B19C7069F4A9
:100B80008150D9F71092DA011092D40106C06C2F6F
:100B90008EEB91E0BCDACC5FE2CFDF91CF9108958C
:100BA000E9E6F0E0808182608083E89A8BE48093BC
:100BB000C9018AE58093C80108952EE088E190E09C
:100BC0000FB6F894A895809360000FBE2093600044
:100BD00084B1876184B93A9A8AB1806E8AB980E01B
:100BE00090E0AFDC80E090E0C0DC80E090E0D9DC19
:100BF00080E090E0DCDC80E090E0BDDCE3DC81E0E4
:100C000090E0A9DCC4E098DCA8952FEB84ED91E09E
:100C1000215080409040E1F700C000002FEB84EDB0
:100C200091E0215080409040E1F700C00000C150A9
:100C300051F747E050E061E070E082EB91E0C0D412
:100C40003FDD82E091E09093F4018093F301909373
:100C5000F6018093F50180E191E0C2D2A1DF539AC1
:100C6000C5E081E090E06DDC2FEB84ED91E0215058
:100C700080409040E1F700C0000080E090E061DC3F
:100C80002FEB84ED91E0215080409040E1F700C0CF
:100C90000000A895C15029F75398DADB7894D8EC76
:100CA000A89533DE80913401E5DB80913401811118
:100CB0001092340180918C01882391F3CD2F25DE91
:100CC0008FE295E70197F1F700C00000C150B9F736
:100CD000E7CFEEE8F1E08FE991E01192E817F9072C
:100CE000E1F70895CF92DF92EF92FF920F931F9357
:100CF000CF93DF9381E090E024DCEBDF80918D01E6
:100D000080938E0110928F018091A0018A3D29F07D
:100D100085E680938F0180E0C1C1EFE9F1E01281A7
:100D200083810481003128F088EC80938F0180E07A
:100D3000B5C1E02EF12CC82FD0E01F920F931F9267
:100D40008F931F921F9381E291E09F938F9337D2ED
:100D50008DB79EB708960FB6F8949EBF0FBE8DBF95
:100D6000113009F055C0C090A401CC202CF486E6C7
:100D700080938F0180E092C18C2D880F3BDC813005
:100D800029F021971C161D063CF014C087E68093BD
:100D90008F015ADC80E082C120E030E0D12CF901E3
:100DA000EB55FE4F808160DCD3942D2D30E02C1765
:100DB0003D07ACF3002349F18C2D880F816042DCA4
:100DC000813021F488E680938F011FC00F2EF0E957
:100DD000CF2EF1E0DF2EF02DC0E0D0E091E0E91A57
:100DE000F108CE15DF0511F051DC01C05CDC8F3F4E
:100DF000EFEF9E0721F488E680938F0106C0F6018D
:100E000081936F012196C01760F31EDC80E046C11C
:100E1000123049F58091A40188232CF486E6809352
:100E20008F0180E03BC1880FE5DB813029F02197FD
:100E30001C161D063CF014C087E680938F0104DC6D
:100E400080E02CC180E090E010E0FC01EB55FE4F0B
:100E500080810ADC1F5F812F90E08C179D07ACF327
:100E6000F3DB80E01BC1133099F5C091A40101119F
:100E700005C086E680938F0180E010C181E090E09C
:100E800060DB8C2F880F8160DDDB813021F488E608
:100E900080938F0117C00F2EF0E9CF2EF1E0DF2EE7
:100EA000F02DC0E0D0E021E0E21AF108CE15DF0518
:100EB00011F0ECDB01C0F7DBF60181936F012196A5
:100EC000C017A0F380E090E03CDBBEDB80E0E6C032
:100ED0001430D9F5EFE9F1E0C5800681CC207CF033
:100EE00000236CF00C1558F010E00C1911090F5F7D
:100EF0001F4F1016110644F0C0E0D0E022C086E675
:100F000080938F0180E0CAC0F12CC0E0D0E0DF2CDC
:100F1000DC0C8D2D880F6EDB81110CC0FE01E257B9
:100F2000FE4FD3822196CF30D10524F088EC8093F8
:100F30008F0107C089DBF3948F2D90E08017910714
:100F400034F3C093900180E0A9C0153031F4809152
:100F5000A40190E000DB80E0A1C0163051F474DB06
:100F600087EB9BE00197F1F700C000002BDB80E0EE
:100F700095C0153619F48091A40190C0163629F455
:100F8000E6DA8093900180E089C01736C9F487E0E3
:100F9000E4EAF1E0A2EBB1E001900D928A95E1F76D
:100FA0008091B60190E09093BA018093B90160916D
:100FB000B701662309F471C080E011DA80E06EC0E9
:100FC000183659F487E0E2EBF1E0A0E9B1E00190D6
:100FD0000D928A95E1F780E061C0193651F4ACDAE0
:100FE00047E050E061E070E082EB91E0F9D280E010
:100FF00055C01A3651F4A0DA47E050E061E070E0E5
:1010000082EB91E0DDD280E049C0143641F481E00A
:10101000809390018CE08093910180E03FC01B366B
:1010200051F48ADA65E580E090E0E3D281E08093D4
:101030008C0180E033C0183C31F48091A40190E031
:10104000B6DA80E02BC0193C29F4B7DA809390011E
:1010500080E024C01A3C29F481E08093340180E0D0
:101060001DC01B3C31F48091A40190E08ADA80E03D
:1010700015C01C3C29F48BDA8093900180E00EC0EF
:101080001D3C31F48091A40190E085DA80E006C037
:1010900086E680938F0180E001C080E090E051DA25
:1010A000DF91CF911F910F91FF90EF90DF90CF9044
:1010B00008951F93CF93DF93C091B001CC23F9F033
:1010C000D62FC61708F4DC2F1091B101212F30E084
:1010D0004D2F50E0BC01C90181569E4F67D01D0FB6
:1010E0001093B101CD1BC093B001C11101C0FADD55
:1010F00081E09091B001992319F080E001C081E076
:10110000DF91CF911F9108951F93CF93DF93D091DB
:10111000B001C62FD61708F4CD2F1091B1014C2F76
:1011200050E0612F70E062577E4F40D01C0F10934B
:10113000B101DC1BD093B0018C2FDF91CF911F91B7
:101140000895FC0120812076203241F522818181A1
:10115000813089F48FEF820F823010F520938D015A
:10116000213011F481E101C083E88093B001109235
:10117000B1018FEF08958930A9F48FEF820F82308B
:1011800098F420938D01213011F481E101C083E8AE
:101190008093B0011092B1018FEF089580E008951F
:1011A00080E0089580E0089580E00895FB01DC016F
:1011B00002C001900D9241505040D8F70895A0E030
:1011C000B0E0E4EEF8E0D9C2FE013596619171918C
:1011D000AF018091F5019091F6012FD0E2E0E9C2D4
:1011E0000F931F93CF93DF93E091F501F091F601F8
:1011F000238121FF1BC0EC0100E010E08991609188
:10120000F5017091F601DB011896ED91FC911997AB
:10121000882331F00995892B89F30FEF1FEFEECF6B
:101220008AE00995892B11F4C80102C08FEF9FEF66
:10123000DF91CF911F910F910895ACE0B0E0E2E211
:10124000F9E08BC27C016B018A01FC0117821682D6
:10125000838181FFB0C1CE0101964C01F7019381DA
:10126000F60193FD859193FF81916F01882309F425
:101270009EC1853239F493FD859193FF81916F0171
:10128000853221F4B70190E0D8D1E8CF512C312C30
:1012900020E02032A0F48B3269F030F4803259F033
:1012A000833269F420612CC08D3239F0803339F4F7
:1012B000216026C02260246023C0286021C027FD51
:1012C00027C030ED380F3A3078F426FF06C0FAE038
:1012D0005F9E300D1124532E13C08AE0389E300DCE
:1012E0001124332E20620CC08E3221F426FD5FC102
:1012F000206406C08C3611F4206802C0883641F4A0
:10130000F60193FD859193FF81916F018111C1CF0A
:10131000982F9F7D9554933028F40C5F1F4FFFE367
:10132000F9830DC0833631F0833771F0833509F0CE
:1013300057C021C0F801808189830E5F1F4F44246C
:101340004394512C540114C03801F2E06F0E711C0B
:10135000F801A080B18026FF03C0652D70E002C0B7
:101360006FEF7FEFC5012C875DD12C0183012C85A8
:101370002F77222E16C03801F2E06F0E711CF80193
:10138000A080B18026FF03C0652D70E002C06FEF22
:101390007FEFC5012C873BD12C012C852068222EA4
:1013A000830123FC19C0832D90E048165906A0F450
:1013B000B70180E290E041D13A94F5CFF50127FCE6
:1013C000859127FE81915F01B70190E036D1311000
:1013D0003A94F1E04F1A51084114510479F7DEC0F4
:1013E000843611F0893631F5F80127FF07C0608196
:1013F0007181828193810C5F1F4F08C06081718170
:10140000882777FD8095982F0E5F1F4F2F76B22E7D
:1014100097FF09C090958095709561957F4F8F4F8C
:101420009F4F2068B22E2AE030E0A40138D1A82EC8
:10143000A81843C0853729F42F7EB22E2AE030E069
:1014400025C0F22FF97FBF2E8F36C1F018F48835F2
:1014500079F0ADC0803719F0883721F0A8C02F2F60
:101460002061B22EB4FE0DC08B2D8460B82E09C051
:1014700024FF0AC09F2F9660B92E06C028E030E0F6
:1014800005C020E130E002C020E132E0F801B7FE03
:1014900007C060817181828193810C5F1F4F06C0FC
:1014A0006081718180E090E00E5F1F4FA401F7D052
:1014B000A82EA818FB2DFF77BF2EB6FE0BC02B2D34
:1014C0002E7FA51450F4B4FE0AC0B2FC08C02B2D28
:1014D0002E7E05C07A2C2B2D03C07A2C01C0752CD2
:1014E00024FF0DC0FE01EA0DF11D8081803311F44F
:1014F000297E09C022FF06C07394739404C0822F12
:10150000867809F0739423FD12C020FF06C05A2C80
:10151000731418F4530C5718732C731460F4B70138
:1015200080E290E02C8789D073942C85F6CF7314D9
:1015300010F4371801C0312C24FF11C0B70180E32B
:1015400090E02C877AD02C8522FF16C021FF03C0A3
:1015500088E590E002C088E790E0B7010CC0822FD8
:10156000867851F021FD02C080E201C08BE227FDA8
:101570008DE2B70190E061D0A51430F4B70180E3AB
:1015800090E05BD05A94F8CFAA94F401EA0DF11DD3
:101590008081B70190E051D0A110F6CF332009F43B
:1015A0005DCEB70180E290E048D03A94F7CFF701E2
:1015B0008681978102C08FEF9FEF2C96E2E1E9C010
:1015C000DC01CB01FC01F999FECF06C0F2BDE1BD03
:1015D000F89A319600B40D9241505040B8F70895F2
:1015E000DC01CB0102C02D9105D041505040D8F70D
:1015F0000895262FF999FECF1FBA92BD81BD20BD57
:101600000FB6F894FA9AF99A0FBE01960895FC0164
:101610000590615070400110D8F7809590958E0F1D
:101620009F1F0895FC016150704001900110D8F790
:10163000809590958E0F9F1F08950F931F93CF93C2
:10164000DF93182F092FEB018B8181FD03C08FEFF2
:101650009FEF20C082FF10C04E815F812C813D81B1
:10166000421753077CF4E881F9819F012F5F3F4FB8
:1016700039832883108306C0E885F985812F099571
:10168000892B29F72E813F812F5F3F4F3F832E8388
:10169000812F902FDF91CF911F910F910895FA0123
:1016A000AA27283051F1203181F1E8946F936E7FA1
:1016B0006E5F7F4F8F4F9F4FAF4FB1E03ED0B4E092
:1016C0003CD0670F781F891F9A1FA11D680F791FD3
:1016D0008A1F911DA11D6A0F711D811D911DA11DE4
:1016E00020D009F468943F912AE0269F11243019F4
:1016F000305D3193DEF6CF010895462F4770405D8F
:101700004193B3E00FD0C9F7F6CF462F4F70405D3D
:101710004A3318F0495D31FD4052419302D0A9F798
:10172000EACFB4E0A6959795879577956795BA9592
:10173000C9F700976105710508959B01AC010A2E58
:1017400006945795479537952795BA95C9F7620F2F
:10175000731F841F951FA01D08952F923F924F92D3
:101760005F926F927F928F929F92AF92BF92CF9231
:10177000DF92EF92FF920F931F93CF93DF93CDB73A
:10178000DEB7CA1BDB0B0FB6F894DEBF0FBECDBFB2
:1017900009942A88398848885F846E847D848C8483
:1017A0009B84AA84B984C884DF80EE80FD800C818C
:1017B0001B81AA81B981CE0FD11D0FB6F894DEBF6F
:0C17C0000FBECDBFED010895F894FFCFDF
:1017CC00FF5A00000003000000006E037F030000BE
:1017DC006C696E6B6D206465627567206D6F6465F6
:1017EC00000A633A256420733A256420723A256412
:0217FC002000CB
:00000001FF
